:0400000007EF00F016
:100008005F8282ED1BF014EF15F0700E846FF0D351
:10001800250E8A19D8B409D06CC0D9FF6DC0DAFF93
:100028008AC0DFFF6C4B6D2BE3D3000E896F000E87
:10003800886F000E8C6F000E8B6F09D08B8705D0F0
:100048008B8103D08C8701D08B856E4B6F2B6EC054
:10005800F6FF6FC0F7FF0800F550200AD8B4F0D7B4
:10006800030AD8B4EFD70E0AD8B4E8D71D0AD8B413
:10007800EBD78BB78B956EC0F6FF6FC0F7FF080004
:10008800F550EFEC1EF0D8A030D0000E896F000EAE
:10009800886F88C060F089C061F0000E636F0A0E37
:1000A800626FA9EC1EF060C088F061C089F06EC074
:1000B800F6FF6FC0F7FF0800F5CF76F0D00E762573
:1000C800776F786BFF0E78237751882778518923CB
:1000D8006E4B6F2B6EC0F6FF6FC0F7FF0800F55030
:1000E800EFEC1EF0D8A015D0D4D76EC0F6FF6FC0C5
:1000F800F7FF0800F5502A0AD8A40BD08451D96E0E
:10010800DA6ADECF88F0DDCF89F0020E84276E4BE5
:100118006F2B6EC0F6FF6FC0F7FF0800F5502E0A70
:10012800D8A437D08C8D6E4B6F2B6EC0F6FF6FC086
:10013800F7FF0800F5502A0AD8A40FD08451D96EC9
:10014800DA6ADF50876F020E842787AF03D0000E6C
:10015800876F8C9D6E4B6F2BD3D0000E876F0ED0A0
:100168000A0E8703F350876F6EC0F6FF6FC0F7FF64
:100178000800F550D00F87276E4B6F2B6EC0F6FF27
:100188006FC0F7FF0800F550EFEC1EF0D8A0B8D00C
:10019800E7D7000E876FB4D08B8DD8D08B8B8B8F21
:1001A800D5D08451D96EDA6ADECF80F0DDCF81F008
:1001B800020E842780518111D8A404D0770E806F55
:1001C8007F0E816F000E836F000E826F03D00001D7
:1001D800824B832B82518025766F83518121776FE3
:1001E80076C0F6FF77C0F7FFF86A070EF76403D00A
:1001F8000800F55005D0F6CFE1FFF7CFE2FFE75052
:100208000009D8A4E4D700018751D8B40ED0800ED5
:1002180087BF7F0E766F8251875D8351800A76593A
:10022800D8B003D087C082F0836B8851825D895132
:100238008359D8B005D08251885F8351895B04D037
:10024800000E896F000E886F8BA709D02BD06CC069
:10025800D9FF6DC0DAFF200EDF6E6C4B6D2B88075F
:10026800D8A089078829F3E18929D8B41BD0EFD70A
:1002780080C0F6FF81C0F7FFF86A6CC0D9FF6DC077
:10028800DAFF070EF76403D00800F55005D0F6CF63
:10029800E1FFF7CFE2FFE750DF6E0001804B812BD3
:1002A8006C4B6D2B8207D8A083078229E1E1832953
:1002B800D8A4DED78BB709D09BD26CC0D9FF6DC04C
:1002C800DAFF200EDF6E6C4B6D2B8807D8A08907EC
:1002D8008829F3E18929D8B48BD2EFD78451D96E14
:1002E800DA6ADF508A6F020E84278A0E806F816B6C
:1002F800000E836F010E826F86D7C00E8B1326D037
:100308006EC0F6FF6FC0F7FF6E4B6F2B0800F5CF7E
:100318008AF08A51000AD8B477D2580AD8B43ED79E
:100328003B0AD8B4DBD7070AD8B410D00D0AD8B422
:100338000DD0060AD8B430D71C0AD8B432D7060A6A
:10034800D8B4DBD70D0AD8B42AD7CFD78BC076F06C
:10035800C00E7617D8A412D08451D96EDA6ADECFCF
:1003680085F0DDCF86F0020E842786AF10D0030E0D
:100378008B13856D861FD8B0862B09D08451D96E12
:10038800DA6ADECF85F0DDCF86F0020E842787514A
:10039800D8A44ED085518611D8A44AD0872B48D0EE
:1003A800010E8A6F050E8A19D8B450D08A51020DF1
:1003B800CF0EF324F66E7C0EF420F76E0900F5508C
:1003C800855D0900F5508659D8A040D08A2BEAD718
:1003D800010E8A6F040E8A19D8B438D08A51020DDA
:1003E800D90EF324F66E7C0EF420F76E0900F55052
:1003F800855D0900F5508659D8A028D08A2BEAD700
:10040800010E8A6F060E8A19D8B420D08A51020DBF
:10041800C30EF324F66E7C0EF420F76E0900F55037
:10042800855D0900F5508659D8A010D08A2BEAD7E7
:100438008B51C00B000AD8B4B3D7400AD8B4E0D760
:10044800C00AD8B4C5D7400AD8B4AAD78A51D88028
:10045800D88487AF875DD8A0D884D8B403D087C0A4
:100468008AF009D08A51D89087AF875DD8B0D880F4
:10047800D8A08AC087F088518911D8B409D08BC018
:1004880076F0030E7617D8B403D08807D8A089076A
:100498008CAD16D0800E87BF7F0E766F8851875D32
:1004A8008951800A7659D8B007D08751885F000EE5
:1004B80087BFFF0E895B04D0000E896F000E886F1E
:1004C800C40E8B15766F080E8C15776F400E761953
:1004D8000CE1080E7719D8A408D088518911D8B42E
:1004E80022D08807D8A089071ED0C00E8B15766F3A
:1004F800080E8C15776F800E761915E1080E77199E
:10050800D8A411D089BF0BD0895104E1030E885DAE
:10051800D8A005D0FE0E8827FF0E892304D0000E30
:10052800896F000E886F8A51766F776B8851765D78
:100538007751800A786F8951800A7859D8B005D0E8
:100548008A51885F000E895B04D0000E896F000E07
:10055800886F8BA54DD08BC076F0030E7617D8B474
:1005680009D06CC0D9FF6DC0DAFF2D0EDF6E6C4B61
:100578006D2B2ED08BA106D06CC0D9FF6DC0DAFFD1
:10058800200EF4D7C00E8B15766F080E8C15776F7A
:10059800800E76191DE1080E7719D8A419D06CC001
:1005A800D9FF6DC0DAFF300EDF6E6C4B6D2B8BBB45
:1005B80004D0000E7B6F780E03D0000E7B6F580EB0
:1005C8007A6F6CC0D9FF6DC0DAFF7AC0DFFFCFD772
:1005D80088518911D8B4F1D06CC0D9FF6DC0DAFF49
:1005E800300EDF6E6C4B6D2B8807D8A08907F0D7CB
:1005F80088518911D8A48BB70FD06CC0D9FF6DC0B2
:10060800DAFF200EDF6E6C4B6D2B8807D8A08907A8
:1006180088518911D8A4F1D78BC076F0030E7617CC
:10062800D8B409D06CC0D9FF6DC0DAFF2D0EDF6ECB
:100638006C4B6D2B08D08BA106D06CC0D9FF6DC058
:10064800DAFF200EF4D7C00E8B15766F080E8C15C6
:10065800776F400E76190DE1080E7719D8A409D0E6
:100668006CC0D9FF6DC0DAFF300EDF6E6C4B6D2B9E
:10067800A4D0C00E8B15766F080E8C15776F800E80
:1006880076191DE1080E7719D8A497D06CC0D9FF48
:100698006DC0DAFF300EDF6E6C4B6D2B8BBB04D058
:1006A800000E7D6F780E03D0000E7D6F580E7C6FA4
:1006B8006CC0D9FF6DC0DAFF7CC0DFFFD7D77DD013
:1006C8008751020DCF0EF324F66E7C0EF420F76EE0
:1006D8000900F5CF62F00A00F5CF63F085C060F03D
:1006E80086C061F081EC1CF060C067F061C068F002
:1006F800000E6A6F0A0E696F66EC1DF0675145D0EF
:1007080085C060F086C061F08751020DD90EF324D0
:10071800F66E7C0EF420F76E0900F5CF62F00A0041
:10072800F5CF63F081EC1CF060510F0B796F8BBB38
:1007380004D09E0E7E6F7E0E03D08D0E7E6F7E0ED1
:100748007F6F79517E25766F000E7F21776F76C097
:10075800F6FF77C0F7FF0800F5CF8AF027D085C0ED
:1007680060F086C061F08751020DC30EF324F66E67
:100778007C0EF420F76E0900F5CF62F00A00F5CF81
:1007880063F081EC1CF06051070B300F8A6F0ED0BC
:100798008B51C00B000AD8B493D7400AD8B4DFD71E
:1007A800C00AD8B4ADD7400AD8B48AD76CC0D9FF2C
:1007B8006DC0DAFF8AC0DFFF59D787078729D8A419
:1007C800E7D78BB789BF14D0895103E18805D8A032
:1007D8000FD06CC0D9FF6DC0DAFF200EDF6E6C4BF6
:1007E8006D2B8807D8A0890788518911D8A4F1D71B
:1007F8006EC0F6FF6FC0F7FF6E4B6F2B0800F5CF8A
:100808008AF08A51D8A404D46CC0D9FF6DC0DAFF2D
:10081800DF6A1200F3C0EAF1F4C0EBF1000E010147
:10082800ED6F000EEC6F000EE96F000EE86F21D23D
:10083800EAC1D9FFEBC1DAFFDF50F26FEA4BEB2BCD
:1008480007D21B0EF219D8A402D0010E76D12B0EB6
:10085800F219D8A402D0020E70D10D0EF219D8B434
:1008680004D00A0EF219D8A4C4D02A510001F75DA9
:1008780001012B510001F859D8B0F8D128A414D09F
:10088800B50E6C6F010E6D6F0C0E6E6F7F0E6F6F75
:10089800F7C070F0F8C071F009EC00F0B50E616FA8
:1008A800010E626F05EC1CF027A61AD0320E01016A
:1008B800436F050E446F3F0E456F550E466FF95155
:1008C800200F476F000E486FBFEC07F0040EE82EAC
:1008D800FED795EC0DF0010E37EC1FF0BFEC07F0DA
:1008E800000E0101F16F000EF06FF7C0EEF1F8C0D5
:1008F800EFF1430E0001606F010E616F000E636F30
:10090800000E626F000E656F400E646F41EC1EF0C2
:10091800200E0101436F10D0EEC1D9FFEFC1DAFFFD
:10092800450EF025E16E010EF121E26EDFCFE7FF03
:10093800EE4BEF2BF04BF12B2A51EE5D2B51EF597B
:10094800D8A0EAD7F851D8B403D0F805D8A40AD06B
:10095800450EF025D96E010EF121DA6E0D0EDF6E0F
:10096800F04BF12BF851D8B404D0020EF819D8A4E2
:100978000AD0450EF025D96E010EF121DA6E0A0E65
:10098800DF6EF04BF12BF051020F446FF7C02AF1E4
:10099800F8C02BF1000E266EBFEC07F0040EE82E0F
:1009A800FED795EC0DF095EC0DF027B027A61BD0DF
:1009B800320E0101436F050E446F3F0E456F550E11
:1009C800466FF951400F476F000E486FBFEC07F0B4
:1009D800100E0001FD6F940EE82EFED7FD2FFCD7F8
:1009E800000095EC0DF0000E0101ED6F010EEC6FAB
:1009F8003DD10001F75101012A5D0001FD6FF85159
:100A080001012B590001FE6FFEBF81D0FE5104E1A8
:100A18003D0EFD5DD8A07BD028A414D0B50E6C6F18
:100A2800010E6D6F670E6E6F7E0E6F6FF7C070F000
:100A3800F8C071F009EC00F0B50E616F010E626F3D
:100A480005EC1CF027A61AD0320E0101436F050EE3
:100A5800446F3F0E456F550E466FF951200F476F93
:100A6800000E486FBFEC07F0040EE82EFED795EC99
:100A78000DF0010E37EC1FF0BFEC07F0000E01017E
:100A8800F16F000EF06FF7C0EEF1F8C0EFF1430E12
:100A98000001606F010E616F000E636F000E626FE0
:100AA800000E656F400E646F41EC1EF0200E0101D0
:100AB800436F10D0EEC1D9FFEFC1DAFF450EF02524
:100AC800E16E010EF121E26EDFCFE7FFEE4BEF2B77
:100AD800F04BF12B2A51EE5D2B51EF59D8A0EAD7F4
:100AE800F051020F446FF7C02AF1F8C02BF1000E45
:100AF800266EBFEC07F0280EE82EFED795EC0DF019
:100B080095EC0DF0000E0101ED6F010EEC6F2AC19E
:100B1800D9FF2BC1DAFFF2C1DFFF01012A4B2B2BD2
:100B2800262AA4D02AC1D9FF2BC1DAFFF2C1DFFFE0
:100B38002A4B2B2B262A000E0101356F97D02B0E3E
:100B4800F219D8A417D0030E356F830E0001606F19
:100B5800010E616F000E636F000E626F000E656F0D
:100B6800320E646F41EC1EF0830E0101246F010EFA
:100B7800256F7CD0000E356FCAD70D0EF219D8B488
:100B880004D00A0EF219D8A45AD024C1D9FF25C11D
:100B9800DAFFDF6A830E0001AC6F010EAD6FFBC098
:100BA800AEF0FCC0AFF0830E0101245D0001B06F10
:100BB800010E010125590001B16F2BEC09F0ACC001
:100BC800E6F1ADC0E7F10101E651E711D8A411D073
:100BD8002AC1D9FF2BC1DAFF2B0EDF6E2A4B2B2B34
:100BE8002AC1D9FF2BC1DAFF2B0EDF6E2A4B2B2B24
:100BF800A2D7FBC064F0FCC065F0FBC060F0FCC08D
:100C080061F021EC1DF06051666FCEEC1EF028A457
:100C180092D7B50E00016C6F010E6D6F480E6E6FA6
:100C28007F0E6F6FFBC070F0FCC071F009EC00F034
:100C3800B50E616F010E626F05EC1CF07CD724C104
:100C4800D9FF25C1DAFFF2C1DFFF244B252B0ED0D7
:100C58003551000AD8B4F5D5010AD8B463D7030AC8
:100C6800D8B46DD7010AD8B488D751D70101E84B59
:100C7800E92B0001F5510101E85D0001F651010180
:100C8800E959D8A0D5D5ECC1F3F0EDC1F4F01200C4
:100C9800000E0001A36F0F0E1A6EA00E196E000E43
:100CA800256E8950200B896E000E8B6EF90E946E9E
:100CB80093689250DF09926E040E206E400E606FAA
:100CC800030E616F000E636F000E626F000E656F9A
:100CD800800E646F41EC1EF02DD1800E256002D08D
:100CE80080B20CD1090E206E09D194929494020E10
:100CF80003D19482070E1A6ED00E196E010EFCD025
:100D080082B002D0030E206E1906D8A01A06195018
:100D18001A10D8A40FD10A0EEFD09492000E80B604
:100D2800010E236E80A60AD0400E2524D96EDA6AF9
:100D3800030EDA228150FF0ADF6E252A28A81AD06E
:100D4800B50E00016C6F010E6D6FFE0E6E6F7D0E9D
:100D58006F6F25C070F0716B80CF72F0736B92CF9C
:100D680074F0756B09EC00F0B50E616F010E626FDF
:100D780005EC1CF0000E80B8010E246E28A847D0A0
:100D88002350D8A415D0B50E00016C6F010E6D6FFD
:100D9800F90E6E6F7F0E6F6F000E716F210E706F00
:100DA80009EC00F0B50E616F010E626F05EC1CF0E6
:100DB8002450D8A419D0B50E00016C6F010E6D6FC8
:100DC800300E6E6F7F0E6F6F8150A16FA26BA11DE9
:100DD800706FA21D716F09EC00F0B50E616F010E06
:100DE800626F05EC1CF013D0B50E00016C6F010E9C
:100DF8006D6F850E6E6F7F0E6F6F8150A16FA26B46
:100E0800A11D706FA21D716F09EC00F0E6D79484E4
:100E1800000E72D082A08ED0050E6ED0949424500D
:100E2800D8A416D0060E206EE80E156E030E166EA8
:100E3800000E176E000E186E27A47CD0400E2524D5
:100E4800D96EDA6A030EDA225EC0DFFF252A72D075
:100E5800020E0101F719D8A44AD73F0E2524D96EEE
:100E6800DA6A030EDA222950DE18D8A440D7060E13
:100E7800206EE80E156E030E166E000E176E000E2D
:100E8800186E58D080A802D0090E206E1506000EE4
:100E9800165A175A185A1550161017101810D8A4A1
:100EA80002D00B0E206E9492949427A643D0320E53
:100EB8000101436F030E446F5F0E456FBFEC07F0EF
:100EC80039D02550D8A428A811D0B50E00016C6FD0
:100ED800010E6D6F530E6E6F7F0E6F6F09EC00F091
:100EE800B50E616F010E626F05EC1CF0010E00017A
:100EF800A36F949294940B0E206E1CD02050000A7D
:100F0800D8B488D7010AD8B4FBD6030AD8B4F1D626
:100F1800010AD8B402D7070AD8B4E7D6010AD8B468
:100F28007DD7030AD8B4AED70F0AD8B4E2D7030ADC
:100F3800D8B4C7D70B0E2018D8A4CFD62550D8B40C
:100F4800120028A61200B50E00016C6F010E6D6F1D
:100F5800520E6E6F7E0E6F6F25C070F0716BA3C05E
:100F680072F0736B09EC00F0B50E616F010E626FE1
:100F780005EC1CF01200000E1F6E020E216E895047
:100F8800200B896E000E8B6E946893689250DF096F
:100F9800926E000E0101386F28A617D0B50E000119
:100FA8006C6F010E6D6FE50E6E6F7E0E6F6F43C135
:100FB80070F0716B44C172F0736B09EC00F0B50E00
:100FC800616F010E626F05EC1CF028AA25D0B50EE2
:100FD80000016C6F010E6D6FE50E6E6F7E0E6F6F08
:100FE80043C170F0716B44C172F0736B09EC00F08F
:100FF800B50E616F010E626F05EC1CF0F60E000174
:101008008D6F7F0E8E6F450E8F6F010E906F44C1EE
:1010180091F0926B8DEC0AF0320E01014319D8A4BD
:1010280010D09296B50E00016C6F010E6D6FF20E26
:101038006E6F7E0E6F6F44C170F0716B09EC00F03B
:1010480010D028A60ED0B50E00016C6F010E6D6F82
:10105800660E6E6F7F0E6F6F44C170F0716B09EC96
:1010680000F028A6CED0B50E0001616F010E626FA8
:1010780005EC1CF0C6D0010E95D0020E93D028A620
:101088001CD0B50E00016C6F010E6D6F7E0E6E6F79
:101098007F0E6F6F430E2124D96EDA6A010EDA22B1
:1010A800DF509D6F9D51706F716B09EC00F0B50EAC
:1010B800616F010E626F05EC1CF0215000019D6FFD
:1010C8009E6BFF0E0101442500019F6FA06BFF0E70
:1010D800A0239D519F191EE19E51A019D8B427A2A3
:1010E80019D0320E01014319D8B414D0929828A609
:1010F80011D0B50E00016C6F010E6D6F360E6E6F5C
:101108007F0E6F6F09EC00F0B50E616F010E626F14
:1011180005EC1CF0430E2124D96EDA6A010EDA229E
:10112800DF50FF0A8A6E212A000E936E030E1DD02F
:10113800A00E156E860E166E010E176E000E186E36
:1011480060D082B20ED01506000E165A175A185AD9
:10115800152857E1162855E1172853E11828D8A46F
:1011680050D0040E1FD09490050E1F6EE1D782B4A4
:101178000ED01506000E165A175A185A152841E1AE
:1011880016283FE117283DE11828D8A43AD0060EC2
:1011980009D093689288948001014451215CD8A0B9
:1011A8006AD7630E1F6E2DD028A6FBD7B50E000197
:1011B8006C6F010E6D6F980E6E6F7F0E6F6F09EC7E
:1011C80000F0B50E616F010E626F05EC1CF0E9D7F7
:1011D8001F50000AD8B44FD7010AD8B44ED7030A13
:1011E800D8B44DD7010AD8B4ACD7070AD8B4BBD7FE
:1011F800010AD8B4BCD7030AD8B4CBD7640AD8B488
:10120800D3D7630E1F18D8A4E3D7320E01014319B0
:10121800D8B492869480946893689250DF09926E4D
:1012280028A611D0B50E00016C6F010E6D6FFB0E74
:101238006E6F7D0E6F6F09EC00F0B50E616F010ED9
:10124800626F05EC1CF0000E0101386F1200B1BF8F
:101258000BD0B15104E1330EB05DD8A005D0000E1B
:10126800AD6F000EAC6F1200ACC0EEF0ADC0EFF089
:10127800B60E606F616B000E636F000E626F000E3A
:10128800656F320E646F41EC1EF0000EF26F000EB7
:10129800F16F1CD0EEC0D9FFEFC0DAFFDF50F06F5E
:1012A800EE4BEF2B0D0EF019D8B41AD00A0EF01928
:1012B800D8B416D0200EF019D8B412D0F151B60F08
:1012C800D96EDA6AF0C0DFFFF14BF22BB051F15D55
:1012D800F251800AB26FB151800AB259D8A0DAD758
:1012E800FA0EEC6F010EED6F200EF019D8B426D06F
:1012F80059D0EEC0D9FFEFC0DAFFDF50F06F200EF3
:10130800F019D8B41BD0F051EFEC1EF0D8A002D0E1
:10131800010E01D0000EB26FF0516DEC1EF0D8A096
:1013280002D0010E01D0000EB211E8A005D0EEC027
:10133800ECF0EFC0EDF026D0EE4BEF2BF151B26F91
:10134800F251B36FF14BF22BB051B25DB351800A39
:10135800B46FB151800AB459D8B014D0CAD7EEC00E
:10136800D9FFEFC0DAFFDF50F06F0D0EF019D8B4D7
:1013780019D00A0EF019D8B415D0F051D8B412D03B
:10138800EE4BEF2BF151B26FF251B36FF14BF22BE1
:10139800B051B25DB351800AB46FB151800AB459EB
:1013A800D8A0DDD7F1C0EAF0F2C0EBF028A41BD03A
:1013B800B50E6C6F010E6D6F390E6E6F7E0E6F6F0E
:1013C800B60E706F716BECC072F0EDC073F0EAC0CE
:1013D80074F0EBC075F009EC00F0B50E616F010E0A
:1013E800626F05EC1CF0000E0001F26F000EF16F49
:1013F800800EB26F020EB36F020EB227000EB32337
:10140800D890F135D96EF235DA6ED890D936DA3609
:10141800B251D926B351DA22DE50DE10D8B41FD724
:10142800800EB26F020EB36FD890F135D96EF235D7
:10143800DA6ED890D936DA36B251D926B351DA22D3
:10144800DECF60F0DDCF61F021EC1DF060C0E8F088
:1014580061C0E9F0800EB26F020EB36FD890F1351B
:10146800D96EF235DA6ED890D936DA36B251D92635
:10147800B351DA22DECF60F0DDCF61F0ACC062F0AC
:10148800ADC063F0E8C064F0E9C065F0C3EC18F0E3
:1014980060516111D8A431D0ACC0A4F0ADC0A5F0A2
:1014A800AEC0A6F0AFC0A7F0ECC0A8F0EDC0A9F0A0
:1014B800800EB26F020EB36F020EB227000EB32376
:1014C800D890F135D96EF235DA6ED890D936DA3649
:1014D800B251D926B351DA2201D80AD00500FA6EE2
:1014E800DE50FD6EDE50FE6EF850FF6EFA501200B0
:1014F800EAC0ACF0EBC0ADF01200F14BF22BF2BF3A
:1015080077D7F25105E1640EF15DD8B0A8D670D74F
:10151800A6D6B50E6C6F010E6D6F7B0E6E6F7E0ECC
:101528006F6F8DC070F08EC071F08FC072F090C078
:1015380073F091C074F092C075F009EC00F0B50E2C
:10154800616F010E626F05EC1CF0000E00019A6FCE
:10155800000E996FE9D0FB0E616F7D0E626F05EC8E
:101568001CF0000E00019C6F000E9B6F31D099C0DB
:1015780093F09AC094F0933B943BF00E94179351D8
:101588000F0B9413F00E931793518F25956F945169
:101598009021966F9B519525D96E9C519621DA6EB4
:1015A800DF50986FB50E6C6F010E6D6F9E0E6E6FEB
:1015B8007F0E6F6F98C070F0716B09EC00F0B50E7C
:1015C800616F010E626F05EC1CF000019B4B9C2BB8
:1015D8009CBF06D09C511FE1100E9B5DD8B01BD05C
:1015E80099C093F09AC094F0933B943BF00E9417F3
:1015F80093510F0B9413F00E93179B5193279C5103
:1016080094239351915D9251800A956F9451800A69
:101618009559D8B0ACD7F20E616F7F0E626F05ECAA
:101628001CF0000E00019C6F000E9B6F58D099C0F3
:1016380093F09AC094F0933B943BF00E9417935117
:101648000F0B9413F00E931793518F25956F9451A8
:101658009021966F9B519525D96E9C519621DA6EF3
:10166800200EDF6429D0B50E6C6F010E6D6FF90E78
:101678006E6F7F0E6F6F99C093F09AC094F0933B92
:10168800943BF00E941793510F0B9413F00E93178D
:1016980093518F25956F94519021966F9B51952565
:1016A800D96E9C519621DA6EDF50976F9751706F03
:1016B800716B09EC00F00AD0B50E6C6F010E6D6FFE
:1016C800460E6E6F7F0E6F6F09EC00F0B50E616FFE
:1016D800010E626F05EC1CF000019B4B9C2B9CBF1C
:1016E80006D09C511FE1100E9B5DD8B01BD099C04D
:1016F80093F09AC094F0933B943BF00E9417935157
:101708000F0B9413F00E93179B5193279C5194231E
:101718009351915D9251800A956F9451800A955921
:10172800D8B085D7994B9A2B9ABF06D09A511BE10E
:10173800500E995DD8B017D099C093F09AC094F024
:10174800933B943BF00E941793510F0B9413F00EA8
:1017580093179151935D9451800A956F9251800A25
:101768009559D8A0F8D6FB0E616F7D0E626F05EC17
:101778001CF0120004013205D8A40ED030511F0B02
:101788000009D8A409D00C8E030E3119D8A402D0B0
:10179800010E01D0000E2F6E3251D8A41200305124
:1017A8001F0B020AD8A4120034510F0B0009D8B439
:1017B800120034510F0B4B6E030E4B601200200EBB
:1017C8003218D8A412000C8E34BF18D034510F0B25
:1017D8004B6E4B50020D0A0EF324D96E010EF42005
:1017E800DA6EDECF50F0DDCF51F034510F0B4B6E77
:1017F8004C6A1E0E4B24D96E010E13D034510F0BB8
:10180800020DF3500F0FD96EDA6ADECF50F0DDCF3C
:1018180051F034510F0B4B6E4C6A210E4B24D96E8C
:10182800010E4C20DA6EDF504F6E4FB006D0FB0E23
:101838005014506EFF0E511404D0040E5010506E08
:101848005150516E34BF0CD034510F0B4B6E4B506E
:10185800020D0A0EF324D96E010EF420DA6E07D0B9
:1018680034510F0B020DF3500F0FD96EDA6A50C0C6
:10187800DEFF51C0DDFF030E3119D8A42AD050C0B5
:10188800D9FF51C0DAFFDFAE17D034BF09D03451C9
:101898000F0B4B6E4C6A1E0E4B24D96E010E08D0EE
:1018A80034510F0B4B6E4C6A210E4B24D96E010E2E
:1018B8004C20DA6E0101DF8250C0D9FF51C0DAFF37
:1018C800000EDB8450C0D9FF51C0DAFF000EDB8E5A
:1018D8001200040E5018506E5150516E50C0D9FF6E
:1018E80051C0DAFFDFAE1BD050C0D9FF51C0DAFFBC
:1018F8007F0EDF1650C0D9FF51C0DAFF000EDB8C17
:10190800000E446E050E436E50C045F051C046F0BF
:10191800000E486E020E476E43EC18F006D050C019
:10192800D9FF51C0DAFF000EDB8C040E5018506E40
:101938005150516E4FB206D050C0D9FF51C0DAFF96
:10194800DFAE2DD0040134BF09D034510F0B4B6EDC
:101958004C6A1E0E4B24D96E010E08D034510F0B61
:101968004B6E4C6A210E4B24D96E010E4C20DA6E58
:101978000101DF9250C0D9FF51C0DAFF3B0EDF16DC
:10198800000E446E050E436E50C045F051C046F03F
:10199800000E486E020E476E43EC18F006D050C099
:1019A800D9FF51C0DAFF3B0EDF16040134510F0B8B
:1019B8004B6E4C6A700E4B244D6E0F0E4C204E6EC3
:1019C8004DC0D9FF4EC0DAFFFE0EDF161200200E02
:1019D800326001D012006DB2120001013B51D8A44F
:1019E80052D0000E0001606F020E616F000E636F2F
:1019F800000E626F000E656F400E646F41EC1EF0C2
:101A0800000E696F020E6A6F400E6B6FE6EC16F0FF
:101A18000001FF6FFF510101F36FF46BF351F411F3
:101A2800D8B431D0000E0001F36F020EF46FF3C189
:101A3800F5F0F4C1F6F0400EF76F020EF86FF3C13F
:101A4800F9F0F4C1FAF0C00EFB6F030EFC6F0EEC58
:101A580004F028A018D0B50E00016C6F010E6D6F50
:101A6800FF0E6E6F7E0E6F6F09EC00F0B50E616FA2
:101A7800010E626F05EC1CF0000E0001616F020E92
:101A8800626F05EC1CF095EC0DF095EC0DF0010182
:101A98003B51D8A443D02650D8A440D0000E256E80
:101AA8004CEC06F02550D8B439D001013B51D8A4EC
:101AB80035D0400E0001646F030E656F25C066F0D7
:101AC800CEEC1EF028A218D0B50E00016C6F010EE6
:101AD8006D6FBD0E6E6F7E0E6F6F09EC00F0B50E68
:101AE800616F010E626F05EC1CF0400E0001616F22
:101AF800030E626F05EC1CF028AA0ED0FC0E000144
:101B08008D6F7F0E8E6F400E8F6F030E906F25C006
:101B180091F0926B8DEC0AF0000E256E95EC0DF0AD
:101B28001200A09A01012E512F11D8B408D02EC14D
:101B3800D9FF2FC1DAFFDFAE02D0A08A1200030E50
:101B48003B19D8A402D0000E3B6F3B51D8A402D059
:101B5800A08A1200020E3B19D8A414D0010E00016D
:101B6800606F000E616F000E626F000E636F020EF1
:101B7800E8EC10F060C02EF161C02FF1030E0101F6
:101B88003B6F62D03B05D8A45FD0400E2A6404D0D6
:101B9800400E00016A6F02D02AC06AF000016A5143
:101BA8002A5C2A6E000E0101186F050E196F6AC0B3
:101BB80069F03A51D8B412D027D01BC1D9FF1CC143
:101BC800DAFF18C1E1FF19C1E2FFDFCFE7FF01012A
:101BD800184B192B1B4B1C2B00016907000169517D
:101BE800D8B416D0EAD71BC1D9FF1CC1DAFF18C177
:101BF800E1FF19C1E2FFDFCFE7FF0101184B192B05
:101C08001B4B1C2B0001690700016951D8A4EBD7B5
:101C18002A50D8A409D0400E6A19D8A402D0020EBE
:101C280001D0030E01013B6F010E0001606F000E31
:101C3800616F050E626F6AC063F0020EE8EC10F087
:101C480060C02EF161C02FF1A08A12003204D8B40E
:101C58006DBA06D0000E686E69806988020E326E11
:101C680068B469A403D06894E1EC1DF06DA202D0B9
:101C7800A19A120068B069A006D04BEC0FF0A08AB8
:101C8800040E326E689068B869A802D014EC1EF091
:101C980068AC1AD069AC0ED0000E446E730E436E59
:101CA800000E456E000E466E000E486E010E476E21
:101CB80043EC18F0689CFFEC1EF02D50D8A42D06BC
:101CC8002D50D8B455EC14F068BA69AA02D087EC44
:101CD8001DF068B269A20FD07F0E446E4368000EF3
:101CE800456E000E466E000E486E010E476E43ECC0
:101CF80018F0000E6A6E040E326002D0A19A12002B
:101D080069A633D0000E536E68A62FD06CCF33F07F
:101D18003330E832E8320F0B2E6E689633B406D0B3
:101D28001E0E2E24D96EDA6A010E05D0210E2E243D
:101D3800D96EDA6A010EDA220101DF702E50D8A4BA
:101D480003D050EC16F00DD0000E446E720E436EA8
:101D5800330E456E466A000E486E000E476E43EC21
:101D680018F0532A030E5364CFD7A19A1200A09AF1
:101D7800000E6A6E000E686E000E706E710E000125
:101D8800606F0F0E616F000E636F000E626F000EC2
:101D9800656F020E646F41EC1EF0160E6F6E9F0E9B
:101DA8006B6E7B0E696E000E686F6851040D000E35
:101DB800F324D96E040EF420DA6EDE6ADE6ADE6A77
:101DC800DD6A682B0B0E6865F0D76D8C000E6E6EA1
:101DD8006D986D9C6896000E0C6E000E046E000ED9
:101DE800066E000E056E68B6F5D7010E0101406F4C
:101DF800010E3F6F000E3E6F000E3D6F000E426FEA
:101E0800000E0001686F6851020DF3500F0FD96E74
:101E1800DA6ADE6ADD6A6851020D0A0EF324D96EA9
:101E2800010EF420DA6EDE6ADD6A210E6825D96EAD
:101E3800DA6A010EDA22DF6A1E0E6825D96EDA6ABE
:101E4800010EDA22DF6A682B020E6865DCD7080EFD
:101E58000F6E040E106E160E706E040E0401036FE2
:101E6800300E026F080E016F040E006F008F000E17
:101E7800346E000E0101146F000E156F000E166F00
:101E8800000E176F000E3C6F000E326E1200A09A03
:101E9800000E6A6E000E686E000E706E710E356E62
:101EA8000F0E366E000E386E000E376E000E3A6E4C
:101EB800020E396E57EC1EF0160E6F6E9F0E6B6E8B
:101EC8007B0E696E000E3D6E3D50040D000EF3242E
:101ED800D96E040EF420DA6EDE6ADE6ADE6ADD6A26
:101EE8003D2A0B0E3D64F0D76D8C000E6E6E6D981A
:101EF8006D9C6896000E0C6E000E046E000E066E49
:101F0800000E056E68B6F5D7010E0101406F010E8F
:101F18003F6F000E3E6F000E3D6F000E426F000EC9
:101F28003D6E3D50020DF3500F0FD96EDA6ADE6A2E
:101F3800DD6A3D50020D0A0EF324D96E010EF4201D
:101F4800DA6EDE6ADD6A210E3D24D96EDA6A010E88
:101F5800DA22DF6A1E0E3D24D96EDA6A010EDA2211
:101F6800DF6A3D2A020E3D64DCD7080E0F6E040EB0
:101F7800106E160E706E040E0401036F300E026FA1
:101F8800080E016F040E006F008F000E346E000EF5
:101F98000101146F000E156F000E166F000E176FFB
:101FA800000E3C6F000E326E1200800E04013019D4
:101FB800D8A41200C00E0C6E78D0940E096E7D0E57
:101FC8000A6E000E0E6E120E0D6E12003251D8A45B
:101FD8003DD03251020DE70EF324F66E7C0EF4204C
:101FE800F76E0900F5CF09F00A00F5CF0AF0020EE6
:101FF8000924356E000E0A20366E35C0F6FF36C04D
:10200800F7FFF86A070EF76403D00800F55005D00B
:10201800F6CFE1FFF7CFE2FFE7500D6E030E09247C
:10202800356E000E0A20366E35C0F6FF36C0F7FF53
:10203800F86A070EF76403D00800F55005D0F6CF0C
:10204800E1FFF7CFE2FFE7500E6E1200000E0C6EB4
:102058001200030E326123D03251020DE10EF32437
:10206800F66E7C0EF420F76E0900F5CF09F00A0031
:10207800F5CF0AF009C0F6FF0AC0F7FFF86A070EA5
:10208800F76403D00800F55005D0F6CFE1FFF7CF8D
:10209800E2FFE750356E35500D6E0E6A1200000EE5
:1020A8000C6E1200000E0C6E12003351010AD8B4E7
:1020B80084D7030AD8B48AD7010AD8B4CAD7F2D7C2
:1020C80020EE01F01D50D9261E50DA22DF50366E60
:1020D8003650055C000E0658D8A005C036F03650BC
:1020E800055E000E065A000E356E0FD0380E3524E8
:1020F800D96EDA6A040EDA2201C0E1FF02C0E2FFFB
:10210800DFCFE7FF014A022A352A3650355CD8A0CE
:10211800EDD705500610D8B432D020EE01F01B5090
:10212800D9261C50DA22080EDF6E20EE02F01B5072
:10213800D9261C50DA22380EDE6E040EDD6E1DC064
:10214800D9FF1EC0DAFFDFBC0DD01BC0D9FF1CC0F1
:10215800DAFF480EDF6E1BC0D9FF1CC0DAFF000E85
:10216800DB8E12001BC0D9FF1CC0DAFF080EDF6E21
:102178001BC0D9FF1CC0DAFF000EDB8E120020EE58
:1021880001F01B50D9261C50DA22080EDF6E20EE13
:1021980002F01B50D9261C50DA22300EDE6E040ED7
:1021A800DD6E1BC0D9FF1CC0DAFF040EDF6E1BC03A
:1021B800D9FF1CC0DAFF000EDB8E049E2C50D8A479
:1021C800120055EC14F01200666F00016051D8B48B
:1021D80007D06651020DF3500F0FD96EDA6A08D096
:1021E8006651020D0A0EF324D96E010EF420DA6E40
:1021F800DECF67F0DDCF68F067516811D8A405D04D
:10220800000E606F000E616F120020EE02F0675141
:10221800D9266851DA2261C0DEFF62C0DDFF20EEF8
:1022280001F06751D9266851DA2263C0DFFF67C021
:10223800D9FF68C0DAFF400EDF1667C0D9FF68C053
:10224800DAFF000EDB8667C0D9FF68C0DAFF000E30
:10225800DB8E6051D8B415D06651020DF3500F0FC4
:10226800D96EDA6ADECF64F0DDCF65F0040E641B48
:10227800000E651B6651020DF3500F0FD96EDA6A16
:1022880018D06651020D0A0EF324D96E010EF420FF
:10229800DA6EDECF64F0DDCF65F0040E641B000E4D
:1022A800651B6651020D0A0EF324D96E010EF42047
:1022B800DA6E64C0DEFF65C0DDFF67C060F068C02D
:1022C80061F012003B6E3550D8B407D03B50020D78
:1022D800F3500F0FD96EDA6A08D03B50020D0A0E80
:1022E800F324D96E010EF420DA6EDECF3CF0DDCF98
:1022F8003DF03C503D10D8A405D0000E356E000EC0
:10230800366E120020EE02F03C50D9263D50DA22FB
:1023180036C0DEFF37C0DDFF20EE01F03C50D92685
:102328003D50DA2238C0DFFF3CC0D9FF3DC0DAFF9C
:10233800400EDF163CC0D9FF3DC0DAFF000EDB8639
:102348003CC0D9FF3DC0DAFF000EDB8E3550D8B453
:1023580015D03B50020DF3500F0FD96EDA6ADECF5D
:1023680039F0DDCF3AF0040E391A000E3A1A3B5014
:10237800020DF3500F0FD96EDA6A18D03B50020DD8
:102388000A0EF324D96E010EF420DA6EDECF39F08E
:10239800DDCF3AF0040E391A000E3A1A3B50020DFE
:1023A8000A0EF324D96E010EF420DA6E39C0DEFF6E
:1023B8003AC0DDFF3CC035F03DC036F012006D98E4
:1023C8000CBE39D004AE0CD0020E306E01013D5166
:1023D800D8B49BEC16F0000E3F6F000E406F120051
:1023E80020EE01F01B50D9261C50DA22080EDF6EB1
:1023F80020EE02F01B50D9261C50DA22300EDE6E79
:10240800040EDD6E1BC0D9FF1CC0DAFF0C0EDF6E98
:102418001BC0D9FF1CC0DAFF000EDB8E0FC0D9FF2E
:1024280010C0DAFF040EDF6E0FC0D9FF10C0DAFF4C
:10243800000EDB8E1200040130AF11D0010E306E99
:1024480001013E51D8B49BEC16F0000E3F6F000E10
:10245800406F2C50D8A4120055EC14F01200020E54
:10246800306E20EE01F01B50D9261C50DA22080EDF
:10247800DF6E20EE02F01B50D9261C50DA22300EF7
:10248800DE6E040EDD6E1BC0D9FF1CC0DAFF040E21
:10249800DF6E1BC0D9FF1CC0DAFF000EDB8E000EFA
:1024A8000101D4D7F9C1AAF0AB6BA6C0D9FFA7C068
:1024B800DAFFDF6AFA0EA81904E1010EA919D8B4E7
:1024C8000AD0A8C066F0A9C067F0BEEC12F066C0DA
:1024D800AAF067C0ABF0320E0101436F060E446FDD
:1024E8003F0E456F350E466F180E476F0001AA5113
:1024F800400F0101486FBFEC07F04CEC06F0255087
:10250800D8A428A41DD0B50E00016C6F010E6D6F04
:10251800200E6E6F7E0E6F6F40C370F0716B09EC0A
:1025280000F0B50E616F010E626F05EC1CF0400EF5
:102538000001646F030E656F010E666FCEEC1EF02E
:10254800320E0101436F050E446F190E456F5F0E81
:10255800466F3F0E476F000E486FBFEC07F0A6C0EE
:10256800D9FFA7C0DAFFDF6A000E0001A56F010ED0
:10257800A46F120002D0664B672B66C0D9FF67C0F4
:10258800DAFF200EDE18D8B4F6D766C0D9FF67C0C8
:10259800DAFF090EDE18D8B4EED7000E6C6F000E05
:1025A8006B6F000E6A6F66C0D9FF67C0DAFF2D0E29
:1025B800DE18D8A402D06A2B08D066C0D9FF67C03D
:1025C800DAFF2B0EDE18D8A41ED0664B672B1BD063
:1025D8006BC060F06CC061F0000E636F0A0E626F32
:1025E800A9EC1EF066C0D9FF67C0DAFFDF50686F3C
:1025F80068516027000E6123D00E60256B6FFF0EB7
:1026080061216C6FE2D766C0D9FF67C0DAFFDF507F
:10261800EFEC1EF0D8B0DCD76A51D8B40DD06BC03F
:1026280068F06CC069F0681F691F684B692B68C047
:1026380066F069C067F012006BC066F06CC067F0A6
:102648001200080E356E0E5010E1080E0D5CD8B061
:102658000CD00DC035F03150D8A402D0010E04D0F2
:102668003104D8A402D0020E316E35500D5E000E32
:102678000E5A20EE01F00F50D9261050DA2235C03C
:10268800DFFF380E0101326F040E336F0CA01CD02F
:102698003AD009C0F6FF0AC0F7FFF86A32C1D9FF7D
:1026A80033C1DAFF070EF76403D00800F55005D0F0
:1026B800F6CFE1FFF7CFE2FFE750DF6E094A0A2ABB
:1026C8000101324B332B35063550D8B41200E1D70F
:1026D80009C0F6FF0AC0F7FFF86A32C1D9FF33C153
:1026E800DAFF070EF76403D00800F55005D0F6CFDF
:1026F800E1FFF7CFE2FFE750DF6E094A0A2A01013E
:10270800324B332B35063550D8B41200E1D70401CB
:102718003039E832030B0009D8A412003CD00C8EE3
:10272800080E326E1200D9EC0FF01200F0EC13F024
:102738001200340E096E0A6A0C80010E0D6E0C8EA2
:102748001200B8EC15F01200BEEC0BF01200E40E0B
:102758003425096E0A6A010E0A220C80010E0D6EDC
:102768000C8E12000C8EE40E3425D96EDA6A010E36
:10277800DA2232C4DFFF1200000E446E020E436EEE
:10278800000E456E000E466E000E486E000E476E37
:1027980043EC18F012003151000AD8B4D2D7010A1C
:1027A800D8B4D2D7020AD8B4CFD7060AD8B4B7D784
:1027B800030AD8B4B8D7010AD8B4DED70F0AD8B4F8
:1027C800B8D7010AD8B4B2D7030AD8B4C0D7010A17
:1027D800D8B4C8D7070A12000C8E710E356E0F0ECA
:1027E800366E000E386E000E376E000E3A6E020E10
:1027F800396E57EC1EF0000E356E040E366E000E64
:10280800386E000E376E000E3A6E300E396E57EC89
:102818001EF06D8C000E4B6E210E4B24D96EDA6AB9
:10282800010EDA22DF6A1E0E4B24D96EDA6A010E17
:10283800DA22DF6A4B2A020E4B64EED7E40E356EBD
:10284800010E366E000E386E000E376E000E3A6EB0
:10285800020E396E57EC1EF06D9C080E0F6E040EBA
:10286800106E000E1D6E040E1E6E1DC01BF01EC0E5
:102878001CF032C434F03450D8A403D0100E326E99
:102888001200000E446E010E436E340E456E466A09
:10289800000E486E010E476E43EC18F0200E326EA3
:1028A800120001014051D8A41200010E406F3F519F
:1028B800D8A41200010E3F6F020E3018D8A414D00D
:1028C80020EE01F00F50D9261050DA22DF6A0FC02F
:1028D800D9FF10C0DAFF480EDF6E0FC0D9FF10C055
:1028E800DAFF000EDB8E12003004D8A41200000EAE
:1028F800416F20EE01F01D50D9261E50DA22080E35
:10290800DF6E20EE02F01D50D9261E50DA22300E5E
:10291800DE6E040EDD6E1DC0D9FF1EC0DAFF040E88
:10292800DF6E1DC0D9FF1EC0DAFF000EDB8E010E60
:10293800416F20EE01F01B50D9261C50DA22080EF8
:10294800DF6E20EE02F01B50D9261C50DA22300E22
:10295800DE6E040EDD6E1BC0D9FF1CC0DAFF800ED0
:10296800DF6E12000FC0D9FF10C0DAFF000EDFBC07
:10297800010E366E040E0F180F6E1050106E080EF2
:102988003218D8A40BD0040132517F0B6E6E6E50F2
:10299800D8B402D0100E01D0040E326E3004D8A480
:1029A8003AD020EE02F00F50D9261050DA22380E15
:1029B800DE6E040EDD6E25EC13F0020E3118D8A47D
:1029C8000DD00FC0D9FF10C0DAFF040EDF6E0FC0A4
:1029D800D9FF10C0DAFF000EDB8E12003650D8A4E3
:1029E8000DD00FC0D9FF10C0DAFF480EDF6E0FC040
:1029F800D9FF10C0DAFF000EDB8E12000FC0D9FF1E
:102A080010C0DAFF080EDF6E0FC0D9FF10C0DAFF62
:102A1800000EDB8E120004BE049E000E306E120003
:102A28005E0EF66E370EF76E000EF86E02EE80F050
:102A380010EE58F00900F5CFEEFFE550E150FAE14D
:102A4800F40EF66E3E0EF76E000EF86E01EEF5F01F
:102A580010EE0AF00900F5CFEEFFE550E150FAE17B
:102A6800100EF66E3F0EF76E000EF86E0900F5CFE9
:102A78005EF003EE00F011EE00F0EE6AE550E15072
:102A8800FCE1E250FAE102EE00F0800EEE6AE806A0
:102A9800FDE101EE00F0E60EEE6AE806FDE104EE67
:102AA80040F0800EEE6AE806FDE100EE01F0340E1B
:102AB800EE6AE806FDE15F905F92000EF86E000195
:102AC80092EF1AF0040130511F0BE806D8A4120047
:102AD8003039E832030BE806D8A412003451D8B4D0
:102AE80032D03405D8A412002ED0D50E096E010EAE
:102AF8000A6E000E0E6E080E0D6E0C800C8E120003
:102B0800D50E096E010E0A6E0C8E120036C405F041
:102B180037C406F0DD0E016E010E026E000E076E60
:102B2800000E086E048E1200DD0E096E010E0A6E8C
:102B3800000E0E6E070E0D6EC10E0C6E120032C422
:102B480039F10C8E12003151000AD8B4CED7010ADF
:102B5800D8B4D6D7210AD8B4D9D7010AD8B4E4D77B
:102B6800030AD8A41200EBD7000E0401386F000E38
:102B7800396F31D00C8E2F04D8A438D0388336D092
:102B88000C8E34D00C8E34BF0CD034510F0B356EF4
:102B98003550020D0A0EF324D96E010EF420DA6EB8
:102BA80007D034510F0B020DF3500F0FD96EDA6AAC
:102BB800DECF36F0DDCF37F036C0D9FF37C0DAFFC9
:102BC800DFAE14D036C0D9FF37C0DAFFDFA40ED08D
:102BD800010E386F0BD030511F0B000AD8B4CAD77A
:102BE800010AD8B4CDD7030AD8B4CCD70CAE12009A
:102BF800380E096E040E0A6E0C80020E0D6E12005D
:102C08003C6E000E3D6E040E3E6E3550366E376AD1
:102C1800D890363637363C50386E396AD8903836C0
:102C28003936D89038363936365038243A6E3750D7
:102C380039203B6ED8903A363B36D8903A363B36F8
:102C48003A503D263B503E223DC0D9FF3EC0DAFFF8
:102C5800DF9E3550D8A409D03C50020D0A0EF3244B
:102C6800D96E010EF420DA6E06D03C50020DF350F6
:102C78000F0FD96EDA6A3DC0DEFF3EC0DDFF3DC0F2
:102C8800D9FF3EC0DAFFDF9C20EE04F03D50D92684
:102C98003E50DA22DF8C12002D0E2D6E33C052F01A
:102CA800FD0E5216D8A43BD033C052F0D890523201
:102CB8003F0E52165250040D000EF3241D6E040EE2
:102CC800F4201E6E1DC01BF01EC01CF0040E1B1845
:102CD8001B6E1C501C6E1DC0D9FF1EC0DAFFDF30F2
:102CE800E8320F0B0D0AD8A417D0300E356E040E3B
:102CF800366E20EE02F01D50D9261E50DA22DECFA5
:102D080037F0DDCF38F0000E3A6E080E396E44EC1D
:102D18001DF02FEC17F0120027EC1BF012003350B7
:102D2800FD0B040AD8A41200B6EC14F01200000E31
:102D38003E6F000E3D6F020E3018D8A41FD020EE53
:102D480001F01B50D9261C50DA22080EDF6E20EE47
:102D580002F01B50D9261C50DA22380EDE6E040E03
:102D6800DD6E1BC0D9FF1CC0DAFF480EDF6E1BC02A
:102D7800D9FF1CC0DAFF000EDB8E12000D500401D3
:102D8800365D0E503759D8B004D036C40DF037C46C
:102D98000EF025EC13F020EE02F00F50D92610505B
:102DA800DA22380EDE6E040EDD6E0FC0D9FF10C0B9
:102DB800DAFF480EDF6E0FC0D9FF10C0DAFF000E31
:102DC800DB8E1200000E2B6E010130513111D8B488
:102DD80006D030C1D9FF31C1DAFFDFBE3AD020EECC
:102DE80001F03051D9263151DA2200016B51DE5CF5
:102DF800D8B00AD0010120EE01F03051D926315166
:102E0800DA22DF5000016B6F000E2B6E0FD0400EE0
:102E18002B24D96EDA6A050EDA222B506925E16E69
:102E2800000E6A21E26EDFCFE7FF2B2A6B512B5C85
:102E3800D8A0EDD7000E606F400E616F050E626F6F
:102E4800400E636F020EE8EC10F060C030F161C014
:102E580031F12B501200000E316E000E2C6E000E58
:102E68003E6F000E3D6F000E416F000E306E0FC0BA
:102E7800D9FF10C0DAFF7F0EDF16040E0F180F6E91
:102E88001050106E0FC0D9FF10C0DAFF7F0EDF168A
:102E9800040E0F180F6E1050106E1BC0D9FF1CC007
:102EA800DAFF7F0EDF16000E0C6E000E0E6E000E9F
:102EB8000D6E000E046E000E066E000E056E8BEC95
:102EC80013F0000E446E030E436E000E456E000EA6
:102ED800466E000E486E000E476E43EC18F0E3ECA9
:102EE80011F01200FA0EA81906E1010EA919D8A4CA
:102EF80002D0000E20D0D20E606F7F0E616FA8C086
:102F080062F0A9C063F0000E656F030E646FC3EC36
:102F180018F060516111D8A402D0010E0CD0A8C0DD
:102F280066F0A9C067F0BEEC12F06651296E295010
:102F3800D8B403D0020E0101F76F320E0101436FBE
:102F4800050E446F3F0E456F550E466FF951400F01
:102F5800476F000E486FBFEC07F0A6C0D9FFA7C0A7
:102F6800DAFFDF6A000E0001A56F010EA46F1200E0
:102F78006DA23AD0010E87EC1FF0120001012C055A
:102F88002D11D8A404D0010E86EC1FF032D04B0EC0
:102F98002C192D11D8A404D0010E87EC1FF029D0CC
:102FA8002D5104E1970E2C5DD8A023D0000E2D6F73
:102FB800000E2C6F1ED001012C052D11D8A404D0B1
:102FC800010E86EC1FF015D0320E2C192D11D8A445
:102FD80004D0010E87EC1FF00CD0B70E2C5D030E49
:102FE8002D59D8B0E3D705D03250200AD8B4C6D767
:102FF800E2D701012C4B2D2B120028A410D0B50EBE
:103008006C6F010E6D6FCB0E6E6F7E0E6F6F09ECDD
:1030180000F0B50E616F010E626F05EC1CF0320E08
:103028000101436F060E446F3F0E456F550E466F04
:10303800F951200F476F040E486F000E496FBFEC1F
:1030480007F0A6C0D9FFA7C0DAFFDF6A28A411D00D
:10305800B50E00016C6F010E6D6FAF0E6E6F7E0EB8
:103068006F6F09EC00F0B50E616F010E626F05EC31
:103078001CF0000E0001A56F010EA46F120017D0FE
:10308800BCEC17F01200BCEC17F0010EBCEC1EF003
:103098001200BCEC17F0020EBCEC1EF01200C5ECDE
:1030A8001AF07FEC1FF0120066EC15F0120043C016
:1030B80049F044C04AF04A50000AD8B404D07F0A04
:1030C800D8A412001AD04950010AD8B4E8D7030A84
:1030D800D8B41200010AD8B4E7D7060AD8B4120047
:1030E800770AD8B41200010AD8B4CAD7070AD8B4E4
:1030F800D0D7010AD8A41200C6D74950FF0A120037
:10310800FA0EA8191AE1010EA919D8A416D027A6F3
:1031180002D0010E01D0000EAA6FAB6BA6C06CF0F6
:10312800A7C06DF0A40E6E6F7F0E6F6FAAC070F00F
:10313800ABC071F009EC00F01DD0A8C066F0A9C0C2
:1031480067F0BEEC12F066C0AAF067C0ABF0AA0543
:10315800AB11D8A404D027500809276E06D02750F1
:10316800F70B276E000E37EC1FF0A6C0D9FFA7C0DB
:10317800DAFFDF6A000EA56F010EA46F12002ED0D1
:1031880060C0F6FF61C0F7FF0800F5500009D8B429
:103198000DD062C0D9FF63C0DAFF60C0F6FF61C01E
:1031A800F7FFDE500900F518D8B414D060C0F6FF58
:1031B80061C0F7FF0800F5CF66F062C0D9FF63C0B1
:1031C800DAFFDF50676F6751665D606F616BD8A08B
:1031D80061071200604B612B624B632B6407D8A018
:1031E80065076429CDE16529D8A4CAD7000E616FA7
:1031F800000E606F1200FA0EA8191AE1010EA91943
:10320800D8A416D027A802D0010E01D0000EAA6FAC
:10321800AB6BA6C06CF0A7C06DF0A40E6E6F7F0EEE
:103228006F6FAAC070F0ABC071F009EC00F019D054
:10323800A8C066F0A9C067F0BEEC12F066C0AAF09C
:1032480067C0ABF0AA05AB11D8A403D0275010096A
:1032580002D02750EF0B276EA6C0D9FFA7C0DAFF10
:10326800DF6A000EA56F010EA46F1200FA0EA819EE
:103278001AE1010EA919D8A416D027A402D0010E6C
:1032880001D0000EAA6FAB6BA6C06CF0A7C06DF0A2
:10329800A40E6E6F7F0E6F6FAAC070F0ABC071F096
:1032A80009EC00F019D0A8C066F0A9C067F0BEEC20
:1032B80012F066C0AAF067C0ABF0AA05AB11D8A49B
:1032C80003D02750040902D02750FB0B276EA6C055
:1032D800D9FFA7C0DAFFDF6A000EA56F010EA46F41
:1032E8001200FA0EA8191AE1010EA919D8A416D0CD
:1032F80027A202D0010E01D0000EAA6FAB6BA6C0A8
:103308006CF0A7C06DF0A40E6E6F7F0E6F6FAAC031
:1033180070F0ABC071F009EC00F019D0A8C066F0ED
:10332800A9C067F0BEEC12F066C0AAF067C0ABF0A7
:10333800AA05AB11D8A403D02750020902D0275000
:10334800FD0B276EA6C0D9FFA7C0DAFFDF6A000E03
:10335800A56F010EA46F1200FA0EA8191AE1010E4A
:10336800A919D8A416D027A002D0010E01D0000EAA
:10337800AA6FAB6BA6C06CF0A7C06DF0A40E6E6F01
:103388007F0E6F6FAAC070F0ABC071F009EC00F04F
:1033980019D0A8C066F0A9C067F0BEEC12F066C0EC
:1033A800AAF067C0ABF0AA05AB11D8A403D0275088
:1033B800010902D02750FE0B276EA6C0D9FFA7C06F
:1033C800DAFFDF6A000EA56F010EA46F1200285005
:1033D800D8B407D0D80E0001616F7E0E626F05EC7D
:1033E8001CF00F0EC112200E896E000E8B6E9468B1
:1033F80093689268928AC70ED56EF294000E256E75
:10340800000E266E000E226E08D0400E2224D96EC1
:10341800DA6A030EDA22DF6A222A7F0E2264F5D7DF
:10342800000E226E08D0430E2224D96EDA6A010EED
:10343800DA22DF6A222A3F0E2264F5D71200F9C188
:10344800AAF0AB6BA6C0D9FFA7C0DAFFDF6AFA0EF5
:10345800A81904E1010EA919D8B40AD0A8C066F0C9
:10346800A9C067F0BEEC12F066C0AAF067C0ABF066
:10347800320E0101436F060E446F3F0E456F550E25
:10348800466F0001AA51200F0101476F080E486FCF
:10349800000E496FBFEC07F0A6C0D9FFA7C0DAFF3E
:1034A800DF6A000E0001A56F010EA46F12002850FC
:1034B800D8B406D0D80E366E7E0E376EAAEC1CF045
:1034C8000F0EC112200E896E000E8B6E94689368E1
:1034D8009268928AC70ED56EF294000E256E000E81
:1034E800266E000E226E08D0400E2224D96EDA6AAB
:1034F800030EDA22DF6A222A7F0E2264F5D7000E35
:10350800226E08D0430E2224D96EDA6A010EDA221E
:10351800DF6A222A3F0E2264F5D71200000E82ECE1
:103528001EF0000E0101386F000E376F2BEC1EF0F5
:103538002850D8B407D03C0E0001616F7F0E626F2F
:1035480005EC1CF0400E0001606F020E616F000E6A
:10355800636F000E626F000E656F400E646F41EC82
:103568001EF0400E01012A6F020E2B6FBBEC0EF00D
:10357800FCEC1DF0080E276EEBEC19F0EBEC0CF0F0
:10358800FDD7000E0101DD6F4B0EDE6F000EDF6F01
:10359800000EE06F000EE16F000EE26F080EE36FA1
:1035A800000E2B6E1A0E3F6E010EC5EC1DF01E0E9E
:1035B8003F6E020EC5EC1DF0000E356E400E366EE5
:1035C800050E376E400E386E020E66EC11F035C0EF
:1035D80030F136C031F1000E01012E6F000E2F6F51
:1035E800000E3B6F1200400E606F020E616F000EFE
:1035F800636F000E626F000E656F400E646F41ECE2
:103608001EF0000E0101356F090E276E000EF86FCF
:103618002A0E5E6E010EF66F2C0EF56F010EF76F17
:10362800400E0001A66F020EA76F000E256E000E59
:10363800266EA6C0D9FFA7C0DAFFDF6A000EA56F05
:10364800010EA46F1200020E3018D8A403D064EC47
:1036580010F01200000E306E4151D8A41FD020EE99
:1036680001F01B50D9261C50DA22080EDF6E20EE1E
:1036780002F01B50D9261C50DA22300EDE6E040EE2
:10368800DD6E1BC0D9FF1CC0DAFF0C0EDF6E1BC03D
:10369800D9FF1CC0DAFF000EDB8E1200000E416F4E
:1036A800120092928092A00E156E860E166E010E72
:1036B800176E000E186E05D01506000E165A175A0A
:1036C800185A1550161017101810D8A4F5D792824A
:1036D8008082A00E156E860E166E010E176E000EF5
:1036E800186E05D01506000E165A175A185A155096
:1036F800161017101810D8B41200F4D70600E1CF2E
:1037080054F0E2CF55F0D9CF56F0DACF57F0F3CFD7
:1037180058F0F4CF59F0F6CF5AF0F7CF5BF0F8CF66
:103728005CF0F5CF5DF02AEC0EF05DC0F5FF5CC0F3
:10373800F8FF5BC0F7FF5AC0F6FF59C0F4FF58C046
:10374800F3FF57C0DAFF56C0D9FF55C0E2FF54C097
:10375800E1FF5F921100BD7FB038B37F6033E27F35
:103768000230D27FEA32E67F5E385D7FF439EA7F45
:103778007432B87F1E3EC27F563EC67F3C3ED67F1F
:10378800FE31AE7F0831247FB637A97FEC2EEE7F5D
:10379800EE356F7FCC3E927FAC24DA7F503BCE7FF4
:1037A8004634DE7F2C3D8C7FA639CA7F0000FA0E96
:1037B800A81913E1010EA919D8A40FD0A6C06CF05E
:1037C800A7C06DF0A40E6E6F7F0E6F6FF5C170F01D
:1037D800F6C171F009EC00F00FD0A8C066F0A9C0DE
:1037E80067F0BEEC12F066C0F5F167C0F6F1A6C04E
:1037F800D9FFA7C0DAFFDF6A000EA56F010EA46F1C
:10380800120015D061C0F6FF62C0F7FFF86A070E14
:10381800F76403D00800F55005D0F6CFE1FFF7CFE5
:10382800E2FFE7505BEC1FF00001614B622B61C0C7
:10383800F6FF62C0F7FFF86A070EF76403D00800C6
:10384800F55005D0F6CFE1FFF7CFE2FFE7500009CA
:10385800D8B41200D7D7FA0EA81912E1010EA91987
:10386800D8A40ED0A6C06CF0A7C06DF0A40E6E6FE1
:103878007F0E6F6FF8C170F0716B09EC00F00ED01D
:10388800A8C066F0A9C067F0BEEC12F0665101014D
:10389800F86FA6C0D9FFA7C0DAFFDF6A000E0001E3
:1038A800A56F010EA46F1200FA0EA81912E1010EFD
:1038B800A919D8A40ED0A6C06CF0A7C06DF0A40EAC
:1038C8006E6F7F0E6F6FF9C170F0716B09EC00F0CD
:1038D8000ED0A8C066F0A9C067F0BEEC12F0665121
:1038E8000101F96FA6C0D9FFA7C0DAFFDF6A000E91
:1038F8000001A56F010EA46F1200000E666F000E86
:10390800656F62516311D8B41CD0010E646F04D086
:10391800D89062376337642B63AFFAD7D89065378E
:1039280066376251605D63516159D8A005D0625114
:10393800605F6351615B6581D89063336233642F44
:10394800EDD765C060F066C061F0120014D036C0D3
:10395800F6FF37C0F7FFF86A070EF76403D00800D0
:10396800F55005D0F6CFE1FFF7CFE2FFE75070EC56
:103978001FF0364A372A36C0F6FF37C0F7FFF86A15
:10398800070EF76403D00800F55005D0F6CFE1FF25
:10399800F7CFE2FFE7500009D8B41200D8D7FA0EE3
:1039A800A81912E1010EA919D8A40ED0A6C06CF06E
:1039B800A7C06DF0A40E6E6F7F0E6F6F28C070F0F9
:1039C800716B09EC00F00DD0A8C066F0A9C067F0D3
:1039D800BEEC12F06651286EA6C0D9FFA7C0DAFF68
:1039E800DF6A000EA56F010EA46F1200FA0EA81967
:1039F80012E1010EA919D8A40ED0A6C06CF0A7C078
:103A08006DF0A40E6E6F7F0E6F6F5EC070F0716BFD
:103A180009EC00F00DD0A8C066F0A9C067F0BEECB4
:103A280012F066515E6EA6C0D9FFA7C0DAFFDF6A42
:103A3800000EA56F010EA46F120060C062F061C095
:103A480063F003D00001624B632B62C0F6FF63C0D2
:103A5800F7FFF86A070EF76403D00800F55005D0A1
:103A6800F6CFE1FFF7CFE2FFE7500009D8A4EAD785
:103A780000016051625D606F61516359616F1200AE
:103A880037C03DF038C03EF035C03BF036C03CF0A2
:103A980010D03DC0D9FF3EC0DAFFDF503F6E3D4A2F
:103AA8003E2A3BC0D9FF3CC0DAFF3FC0DFFF3B4A9C
:103AB8003C2A3906D8A03A063928EBE13A28D8B486
:103AC8001200E7D769516A11D8B418D0010E6B6F8C
:103AD80004D0D89069376A376B2B6AAFFAD7695127
:103AE800675D6A516859D8A004D06951675F6A5107
:103AF800685BD8906A3369336B2FF1D767C067F07A
:103B080068C068F0120070A01DD01DC0D9FF1EC08B
:103B1800DAFF800EDE18D8A414D00FC0D9FF10C069
:103B2800DAFF840EDE18D8A40CD01DC0D9FF1EC041
:103B3800DAFF0C0EDF6E1DC0D9FF1EC0DAFF000EC3
:103B4800DB8E7090689A1200000EAB6F010EAA6FA0
:103B580080A404D0000EAB6F000EAA6FA6C06CF054
:103B6800A7C06DF0A40E6E6F7F0E6F6FAAC070F0C5
:103B7800ABC071F009EC00F0000EA56F010EA46F48
:103B88001200426E3FA405D0000E356E425004EC80
:103B980016F03FA205D0010E356E425004EC16F027
:103BA800700E4224406E416A0F0E412240C0D9FF78
:103BB80041C0DAFF3FC0DFFF1200000E0101426F73
:103BC800000E446E740E436E000E456E000E466E77
:103BD800000E486E000E476E43EC18F06D92699423
:103BE80001D0689468B4FDD7000E01013C6F120043
:103BF8003250D8A41200000E6D6E000E696E160EBB
:103C08006F6E9F0E6B6E7B0E696ED08EA28AA08A35
:103C1800F28E01D06D866DA6FDD7010E326E1200B0
:103C2800698468986D82010E0101426F000E3C6F35
:103C3800000E446E750E436E000E456E000E466E05
:103C4800000E486E000E476E43EC18F012000C0E82
:103C5800AF6E000EB06EB896AC98AB8EAB88AB9AD0
:103C68009D989D9AD08E9F8AF28EAC90AB9CAC9A10
:103C7800AC8AAC94000E346F120060C066F061C06C
:103C880067F008D066C0D9FF67C0DAFF62C0DFFFFF
:103C9800664B672B6407D8A065076429F3E165299B
:103CA800D8B41200EFD735C03BF036C03CF008D08E
:103CB8003BC0D9FF3CC0DAFF37C0DFFF3B4A3C2A94
:103CC8003906D8A03A063928F3E13A28D8B41200C0
:103CD800EFD7656F010E0001646F7B0E656103D03D
:103CE800610E656107D06551DFEC1EF0D8B002D0D7
:103CF800000E646F64C063F0633112000001606FEE
:103D080007D0010E82EC1FF0010E83EC1FF01200A9
:103D180000016051000AD8B4F4D7010AD8B41200DF
:103D2800030A1200A6C06CF0A7C06DF0AA0E6E6F51
:103D38007D0E6F6F180E706F7F0E716F09EC00F0BB
:103D4800000EA56F010EA46F120060516203F3CF3D
:103D580064F0F4CF65F060516303F3506527615157
:103D68006203F350652764C060F065C061F012001B
:103D7800356E07D0010E84EC1FF0010E85EC1FF0A4
:103D880012003550000AD8B4F5D7010AD8B4120089
:103D9800030A1200A09A01013B51D8A40AD064C0BA
:103DA8001BF165C01CF166C02AF0010E3A6F010EC6
:103DB8003B6FA08A1200626F000E0001616F5B0EFC
:103DC800626105D0400E626502D0010E616F61C06C
:103DD80060F060311200626F000E0001616F3A0EF0
:103DE800626105D02F0E626502D0010E616F61C05D
:103DF80060F060311200010E01011427000E152336
:103E0800162317234251D8A412003C2B3C51D8A4A6
:103E180012003C691200A6C06CF0A7C06DF0D80E65
:103E28006E6F7D0E6F6F09EC00F0000EA56F010E2E
:103E3800A46F1200000E37EC1FF0A6C0D9FFA7C070
:103E4800DAFFDF6A000EA56F010EA46F120055ECB1
:103E58001BF0A6C0D9FFA7C0DAFFDF6A000EA56F66
:103E6800010EA46F12000001606F00016005D8A464
:103E780003D0929A809A1200928A808A1200ABA28A
:103E880004D0AC9AAC8AAB98AB88ABA41200AE5005
:103E9800AC9AAC8A1200ABA204D0AC9AAC8AAB98AC
:103EA800AB88ABA41200AE50AC9AAC8A12000001E9
:103EB800606F03D043EC1FF004009EA8FBD760C0DE
:103EC800ADFF1200A6C0D9FFA7C0DAFFDF6A000E57
:103ED800A56F010EA46F1200356E03D04FEC1FF0D2
:103EE80004009EA8FBD735C0ADFF12002C010103CA
:103EF800144E554C4C005BEC1AF0120012001200E4
:093F080012001200120012002A3E
:107CC2000001000800400000020010008001000ACC
:107CD200006400E80310270100100000010010A654
:107CE2007D607D2C7DE97C09024300020100C032E7
:107CF200090400000102020100052400100104240D
:107D02000202052406000105240100010705810382
:107D120008000209040100020A000000070502022D
:107D22004000000705820240000034034300440083
:107D320043002000520053002D0032003300320075
:107D4200200045006D0075006C0061007400690040
:107D52006F006E002000440065006D006F00340368
:107D62004D006900630072006F00630068006900E3
:107D72007000200054006500630068006E006F0010
:107D82006C006F0067007900200049006E006300FC
:107D92002E001201000202000008D8040A000001AD
:107DA20001020001040309045072656C6F6769786F
:107DB20020475049422D55534220436F6E74726FD3
:107DC2006C6C65722076657273696F6E20362E3325
:107DD2002025730D0A004E6565642068656C703F4E
:107DE200204C6F6F6B20696E2074686520736F750D
:107DF20072636520636F6465210D0A0020677069F4
:107E0200625F7074723A20256420706F7274613AF6
:107E12002025582074726961733A202558000D0A92
:107E220053706F6C6C207374617475732062797413
:107E3200653A20255820000D0A636F6D6D616E64EE
:107E42003A202573202573206C656E20256420005E
:107E52000D0A52583A2025642074696D656F757455
:107E620020256420000D0A64756D70696E672064B8
:107E72006174613A20257320000D0A44756D7020EB
:107E820025732025582025580D0A0030313233340D
:107E92003536373839414243444546003031323372
:107EA2003435363738396162636465660020657837
:107EB2006974696E6720636C7220000D0A46726FE6
:107EC2006D20475049423A200020696E736964650B
:107ED20020636C722000475049425F496E697428E2
:107EE2002920000D0A54583A2025582025582000F0
:107EF200434D44206C656E3A20256420000D0A46ED
:107F0200726F6D205553423A20000D0A646174610C
:107F12003A20257320004D617220323520323032F2
:107F22003400726561645F746D6F5F6D73005B2511
:107F32003032585D3C454F493E005374617274695A
:107F42006E672E2E2E007265706C793A2025732092
:107F5200002074696D656F75742000656F745F63CE
:107F62006861720044415441206C656E0073617611
:107F72006563666700286E756C6C29003C2530329B
:107F8200583E005B253032585D00646562756700BB
:107F920073706F6C6C003C4552523E0020253032AB
:107FA200580025640D0A0072656164006D6F646596
:107FB200006175746F0068656C70006164647200C2
:107FC200696663006C6F6300656E640074726700BB
:107FD200656F69006C6F6E00737271007665720076
:107FE200636C7200656F7300656F74007273740066
:0E7FF200207C200054580025630052580000E7
:020000040020DA
:08000000FFFFFFFFFFFFFFFF00
:020000040030CA
:0E000000240E3F1EFF8181FF0FC00FE00F4056
:00000001FF
